:100000000C941E060C9444280C9471280C944606FB
:100010000C9446060C94E9120C9446060C94460681
:100020000C9446060C9446060C9446060C94460620
:100030000C9446060C9446060C9446060C94460610
:100040000C949E280C9446060C948C2C0C94CF2C6B
:100050000C9446060C9446060C9446060C944606F0
:100060000C9446060C944606AB180D19EC18EF18C4
:10007000F218F518F818FB18FE180D1907193F1A91
:10008000411A411A3F1A411A411A411A411A411A9A
:10009000411A411A411A411A411A411A411A411A88
:1000A000C519411A411A411A411A411A3619411A01
:1000B000411A411A411A411A411A411A411A411A68
:1000C000411A411A411A411A411A411AD119D1193A
:1000D000D119D119D119D119D119D119D119411A5F
:1000E000411A411A411A411A411A3619D019D01928
:1000F000D019D019411ADE19E419EA19F019F619C4
:10010000FC19021A081A121A1C1A261A301A771920
:100110003919411A411A411A411AC519411A411A8D
:10012000411A411A411A411A411A411ACF19CF19DD
:10013000CF19CF19411ADE19E419EA19F019F61985
:10014000FC19021A081A121A1C1A261A301A7719E0
:100150003919411A411A411A411AC519741A741AE7
:10016000741A741A741A741A741A741A741A741A1F
:10017000741A741A741A8B1B8B1B8B1B8B1B8B1B97
:100180008B1BB91AC31ACD1AD71A351B3F1B4E1B2E
:100190005F1BE71CFC1C081D111D201D451D4E1D6D
:1001A000971D601DA920AF20B520BC20CA20EC20DF
:1001B0000A21456E746572206D656E752E2E2E00B7
:1001C000546F67676C6564206D6963726F50504D42
:1001D00000546F67676C656420696E76657274653C
:1001E000642050504D2100546F67676C6564205443
:1001F00058206D7574696E672100546F67676C6570
:10020000642074656C656D65747279210050726F3D
:10021000746F636F6C206572726F72207769746897
:100220002052580054696D656F7574207768656E4B
:1002300020636F6E6E656374696E6720746F205201
:100240005800507265737320616E79206B65792058
:10025000746F2063616E63656C00436F6E6E6563DF
:1002600074696E6720746F2052582C20706F776508
:100270007220757020746865205258202877697440
:10028000682062696E6420706C7567206966206EF4
:100290006F74207573696E6720616C776179732064
:1002A00062696E642900546F67676C656420276912
:1002B0006D6D656469617465206F75747075742700
:1002C00000546F67676C65642027736C61766520E6
:1002D0006D6F64652700546F67676C6564202761E4
:1002E0006C776179732062696E642700546F676769
:1002F0006C65642050504D206368616E6E656C20A3
:100300006C696D69740053657420525353492069B8
:100310006E6A656374696F6E206368616E6E656C8A
:100320002028303D3D64697361626C652900536526
:10033000742050504D206D696E696D756D20737914
:100340006E630053657420626561636F6E20696E31
:1003500074657276616C0053657420626561636FC9
:100360006E2064656C617900536574206265616319
:100370006F6E206672657175656E637920696E2097
:10038000487A3A20303D64697361626C652C205074
:10039000783D504D52206368616E6E656C20782CFC
:1003A0002046783D465253206368616E6E656C202E
:1003B00078005365742050574D2073746F7020641B
:1003C000656C61792028302064697361626C6564B2
:1003D0002C20312D323535203D3D20302E317320FB
:1003E0002D2035306D696E29005365742050504DB5
:1003F0002073746F702064656C61792028302064EC
:10040000697361626C65642C20312D323535203D75
:100410003D20302E3173202D2035306D696E29003E
:10042000536574206661696C736166652064656CF0
:1004300061792028302064697361626C65642C20C6
:10044000312D323535203D3D20302E3173202D2089
:1004500035306D696E29002A2A2A2A2A2A2A2A2A50
:100460002A2A2A2A2A2A2A2A2A2A2A2A2A2A2A2AEC
:100470002A2A2A2A0052582041636B6564202D20C5
:1004800072657665727420737563636573736675E0
:100490006C21002A2A2A2A2A2A2A2A2A2A2A2A2AAD
:1004A0002A2A2A2A2A2A2A2A2A2A2A2A2A2A2A2AAC
:1004B000002A2A2A2A2A2A2A2A2A2A2A2A2A2A2AC6
:1004C0002A2A2A2A2A2A2A2A2A2A2A2A2A2A00528E
:1004D000582041636B6564202D20757064617465DC
:1004E000207375636365737366756C21002A2A2A0D
:1004F0002A2A2A2A2A2A2A2A2A2A2A2A2A2A2A2A5C
:100500002A2A2A2A2A2A2A2A2A2A0056616C696457
:100510002063686F69636573206172653A205B319F
:100520005D2D5B31365D20286368616E6E656C20E1
:10053000312D31362900536574206F7574707574D0
:1005400020666F7220706F727420005B585D2061AE
:10055000626F7274206368616E67657320616E6498
:10056000206578697420525820636F6E6669670051
:100570005B535D20736176652073657474696E6783
:100580007320746F205258005B525D20726576654F
:1005900072742052582073657474696E6773207486
:1005A0006F2064656661756C747300557365206EA9
:1005B000756D62657273205B312D445D20746F2010
:1005C0006564697420706F727473205B452D515D92
:1005D00020666F722073657474696E677300202DD6
:1005E00020726563656976657220636F6E66696700
:1005F000757261746F722C20727820737720000AF4
:100600000A6F70656E4C52536E67200053657420FC
:1006100073657269616C2062617564726174653AB8
:10062000200056616C69642063686F696365733A82
:100630002031202D20342B34202F2032202D203823
:10064000202F2033202D20382B34202F2034202D14
:10065000203132202F2035202D2031322B34202FF5
:100660002036202D20313600536574204368616E9A
:100670006E656C20636F6E6669673A20005365741F
:100680002044617461726174652028302D32293AEA
:10069000200053657420486F70206368616E6E653A
:1006A0006C7320286D61782032342C207365706162
:1006B000726174656420627920636F6D6D61732966
:1006C0002076616C69642076616C75657320312DCC
:1006D0003235353A2000536574206368616E6E656B
:1006E0006C2073706163696E6720287831306B48C5
:1006F0007A293A200053657420524620706F77653E
:10070000722028302D37293A200053657420524634
:10071000206D6167696320286865782920652E67E8
:100720002E20307844454144463030443A2000532E
:1007300065742062617365206672657175656E63AC
:10074000792028696E20487A293A20005B5A5D207A
:10075000656E746572207265636569766572206383
:100760006F6E66696775726174696F6E2075746902
:100770006C79005B465D20646973706C61792061FF
:10078000637475616C206672657175656E63696509
:10079000732075736564005B525D2063616C6375E3
:1007A0006C6174652072616E646F6D206B65792079
:1007B000616E6420686F70206C697374005B495DC2
:1007C000207265696E697469616C697A6520736508
:1007D0007474696E677320746F20736B65746368DB
:1007E0002064656661756C7473005B585D2072658A
:1007F00076657274206368616E67657320616E64EC
:100800002065786974206D656E75005B535D20739B
:100810006176652073657474696E677320746F20E8
:10082000454550524F4D20616E64206578697420B3
:100830006D656E7500557365206E756D62657273BA
:10084000205B302D395D20746F20656469742070E1
:100850006172616D657465727300202D2053797328
:1008600074656D20636F6E66696775726174696F18
:100870006E000A0A6F70656E4C52536E672000510D
:1008800029204F7574707574206265666F726520DB
:100890006C696E6B20283D465329203A2000502970
:1008A00020536C617665206D6F64652028657870D3
:1008B0006572696D656E74616C293A20004F29205C
:1008C00054696D65642042494E44206174207374FC
:1008D000617274757020203A20004E292050504DCE
:1008E000206F7574707574206C696D69746564200F
:1008F000202020203A200044495341424C454400E6
:100900004D292050504D205253534920746F20637D
:1009100068616E6E656C202020203A20004C2920F2
:1009200050504D206D696E696D756D2073796E63E1
:10093000202875732920203A200044495341424C15
:100940004544004B29204661696C736166652062ED
:100950006561636F6E20696E74762E2028312D32AA
:10096000353573293A20004A29204661696C736144
:10097000666520626561636F6E2064656C617920D5
:1009800028302D323535203D3E20313073202D204A
:100990003135306D696E293A200049292046616958
:1009A0006C7361666520626561636F6E206672714B
:1009B0002E203A200048292050574D2073746F7024
:1009C0002064656C6179202020202020203A2000BE
:1009D00047292050504D2073746F702064656C61FE
:1009E00079202020202020203A200046292046611E
:1009F000696C736166652064656C617920202020D4
:100A00002020203A200050574D206368616E6E65AB
:100A10006C200066756E6374696F6E3A2000292041
:100A2000706F72742000506F776572546F776572C3
:100A300000445446205548462033322D62697420C4
:100A400031306368004F70656E4C52536E67525878
:100A5000206D696E6920342F36636800466C7974A6
:100A6000726F6E2F4F72616E6765525820554846FF
:100A70002038636800525820747970653A20004429
:100A8000697361626C656400487A00203D3D200016
:100A900043616C63756C61746564207061636B6540
:100AA0007420696E74657276616C3A200042292068
:100AB0004D6963726F202868616C66292050504D23
:100AC000202020203A00412920496E766572746505
:100AD000642050504D20696E20202020203A0030A4
:100AE00029204D7574652062757A7A657220286DAB
:100AF0006F73746C79293A003929205365726961E2
:100B00006C2062617564726174653A00736D617224
:100B100074506F7274004672536B79005472616E38
:100B200073706172656E740044697361626C6564B0
:100B30000038292054656C656D657472793A2020FF
:100B40002020202020003729204368616E6E656CCC
:100B500020636F6E6669673A202000362920446161
:100B60007461726174652028302D32293A2020206A
:100B700000352920486F70206368616E6E656C7364
:100B80003A2020202020003429204368616E6E65C1
:100B90006C2073706163696E673A202000332920EE
:100BA000524620706F7765722028302D37293A2001
:100BB0002020003229205246206D616769633A2067
:100BC0002020202020202020003129204261736530
:100BD000206672657175656E63793A202020000089
:100BE00000000700020100000304060000000000EE
:100BF00000000001020408102040800102040810D7
:100C00002001020408102004040404040404040263
:100C10000202020202030303030303000000002395
:100C2000002600290000000000250028002B0000FD
:100C3000000000240027002A0000BD2D11241FBE43
:100C4000CFEFD8E0DEBFCDBF13E0A0E0B1E0E8E831
:100C5000F1E602C005900D92A83CB107D9F716E065
:100C6000A8ECB3E001C01D92AC38B107E1F71CE07D
:100C7000CCE3DCE004C02297FE010E94C62ECA33FA
:100C8000D107C9F70E94F92D0C94C2300C940000D2
:100C900080917105813019F482E080937105809113
:100CA0007105833019F484E0809371050895A89547
:100CB0000895DC01ED91FC910190F081E02D099502
:100CC00008952091720530917305382748E0C901D5
:100CD000880F991F37FF06C09C0151E2252750E17C
:100CE000352701C09C01415091F730937305209343
:100CF0007205089588E38093740580E092ECA1E08A
:100D0000B0E08093750590937605A0937705B09336
:100D1000780587E08093810580EC92E9ADEEB9E13A
:100D20008093790590937A05A0937B05B0937C0519
:100D300085E0809382058DEE9EEFADEABEED809357
:100D40007D0590937E05A0937F05B0938005E3E831
:100D5000F5E080E090E0863028F4DC01AE54BC4F32
:100D60002C9101C020E0219301968831910599F7DB
:100D700082E080939B058AE080939C05089580EC37
:100D800091EDA8E9BBE18093B9059093BA05A093D2
:100D9000BB05B093BC0580E090E0A0E0B0E5809397
:100DA000BD059093BE05A093BF05B093C005E1ECCF
:100DB000F5E080E081938F5F8031E1F70895A0E056
:100DC000B0E0E5EEF6E00C948F2ED82F0E94F428C8
:100DD0006115710581059105C9F30E94322F1092AA
:100DE0007D0510927E0510927F0510928005C4E06B
:100DF000812C912C54018A94C0907D05D0907E0561
:100E0000E0907F05F0908005FE2CED2CDC2CCC24AE
:100E10000E942D2FA50194010E946E2E6C0D7D1D48
:100E20008E1D9F1D60937D0570937E0580937F05C9
:100E300090938005C15001F7DD2309F450C003E809
:100E400015E0E801A12CB12C62E3C62ED12CE12CD7
:100E5000F12C8881882309F442C0B39419F40E94CC
:100E60007A063DC00E942D2FA70196010E946E2E8A
:100E7000E1E0E60FA3E8B5E08A2F801B8A1520F495
:100E80008D918E13F9CFE9CF2091820530E0A0E15A
:100E9000B7E20E94062E9B01AC01AE2FB0E00E948B
:100EA000152E4090790550907A0560907B057090E2
:100EB0007C05640D751D861D971D4090B9055090E9
:100EC000BA056090BB057090BC05461657066806CB
:100ED000790618F2E993A39488E1A812BACFCDB7A6
:100EE000DEB7E0E10C94AB2E8436910520F4BC0112
:100EF00080E090E017C09C018E3B910528F42A55B4
:100F00003109AAE0B0E00CC0823D910528F4245BD1
:100F10003109A4E6B0E004C02D5C3109A8E5B2E0D7
:100F20000E94062EA4E6B0E09B01AC010E94152EA3
:100F3000089590E08C599F4F0E947407089561E0D6
:100F40008AE00E94A12960E08AE00E94DA290895DF
:100F5000892B11F061E001C060E08AE00E94DA298B
:100F6000089560E089E00E94A12961E088E00E9484
:100F7000A12961E087E00E94A12960E082E00E944F
:100F8000A12961E084E00E94A129089542E050E097
:100F900068E476E080E00E9424280895E3E0F0E031
:100FA00089E080935700E491E67081E0E63009F033
:100FB00080E00895CF93DF93C82F0E94CE07882347
:100FC00081F0DFB781E080937005F8940E945706A6
:100FD00088E180936000C0936000C1110E945706B1
:100FE000DFBFDF91CF9108958F929F92AF92BF9212
:100FF000CF92DF92EF92FF92CF93FC01C0A5EC2F2E
:10100000E770F0E0E658FC4FA081B0E0C7FF03C0F6
:1010100024E130E002C02FE030E0FC0197A183E141
:10102000989FF0011124E25CFE4F80809180A280A5
:10103000B380A20FB31F20E43FE14DE750E00E94D0
:10104000202EA50194010E944C2E8C2F887149F40A
:1010500069017A01E0EDCE0EE7E0DE1EE11CF11C35
:101060001BC0C7FF05C060E47AE88CE29EE004C0C4
:1010700060E07EEE8AEB9BE069017A01F8EBCF0E2F
:10108000FBE0DF1EE11CF11CA50194010E944C2E27
:10109000C20ED31EE41EF51EC701B60169517C4F76
:1010A0008F4F9F4F28EE33E040E050E00E944C2EDF
:1010B000A8EEB3E00E94152ECF91FF90EF90DF9045
:1010C000CF90BF90AF909F908F9008958F3F9105E4
:1010D00051F048F0811522E0920738F081159340D5
:1010E00030F482E0089580E0089581E0089583E07F
:1010F0000895A0E0B0E0EFE7F8E00C94982EEB0143
:101100008A01B82FB695A0E028813981F8012083A3
:101110002A813B8121832C813D8122832E813F8145
:101120002383688179814A815B812C813D81EE81B5
:10113000FF819F2F9295990F990F907C272F2370F5
:10114000922B252F2370220F220F922B232F2370F7
:101150002295207F922BF80194830B5F1F4F2896D6
:10116000AF5FBA1788F680FF24C0888199810E94FA
:101170006608D82E8A819B810E946608E82E8C81A1
:101180009D810E946608F82E8E819F810E946608CC
:10119000F0E4DF9EA001112490E1E99E900111246A
:1011A000242B282BE4E0FE9EB0011124262BF8010D
:1011B0002083CDB7DEB7E7E00C94B42E803223E075
:1011C000920708F1883E23E0920740F48F51934044
:1011D000E4E096958795EA95E1F70895803D27E04C
:1011E000920718F48C5D93400895883928E092079F
:1011F00068F4885C974074E0969587957A95E1F756
:101200008D509C4F089580E090E008958FEF93E01B
:1012100008958C30910540F4A4E0880F991FAA9599
:10122000E1F7885D9C4F0895843F23E0920718F40E
:1012300084529C4F0895811524E0920740F486570C
:10124000934FF4E0880F991FFA95E1F7089580E92C
:1012500098E008959C013695279525753575821B74
:10126000930B9C0123733373969587959695879579
:1012700083739373820F931F9C0154E036952795D7
:101280005A95E1F7280F391F2F703F7041E051E068
:10129000249FC001259F900D349F900D1124892F0C
:1012A00008955F98882319F00000289A02C0000072
:1012B000289800005F9A000008955F9A000083B1AB
:1012C0005F980000869581700895CF93DF93D82FA3
:1012D0005C9A5F985C98C8E08D2F80780E945109D5
:1012E000DD0FC150C9F75F98DF91CF9108958F77D7
:1012F0000E9465090895CF93DF93D82FC8E08D2F02
:1013000080780E945109DD0FC150C9F75F98DF91C5
:10131000CF910895CF93DF935F98C8E080E0D82FF6
:10132000DD0F0E945D098D0FC150C9F7DF91CF918C
:1013300008950E9477090E948A095C9A0895A1E0A5
:10134000B0E0E5EAF9E00C949D2E806869830E9484
:1013500065096981862F0E947B095C9A2196E2E0EB
:101360000C94B92ECF93C0917D05C827E82FF0E0EB
:10137000EC58FA4F678589E70E949F096C2F8DE32F
:101380000E949F096C2F82E40E949F09CF910895CB
:1013900086E20E9499090895CF93DF93EC016C8156
:1013A0008CE10E949F096D818DE10E949F096E81F1
:1013B0008EE10E949F096F8180E20E949F096885EB
:1013C00081E20E949F09698582E20E949F096A85E5
:1013D00083E20E949F096B8584E20E949F096C85CD
:1013E00085E20E949F096D858AE20E949F096E85B1
:1013F0008EE60E949F096F858FE60E949F0968898B
:1014000080E70E949F09698981E70E949F096A8994
:1014100082E70E949F09DF91CF910895CF92DF92DA
:10142000EF92FF92CF93DF936B017C01C11488E3AD
:10143000D8068CE9E8068CE1F80628F5C701B60164
:1014400020E836E948E950E00E944C2EE90168970F
:1014500060E879E687E69FEF0E94282E6C0D7D1DDF
:101460008E1D9F1DF2E0660F771F881F991FFA954A
:10147000D1F721E732E040E050E00E944C2EF22EFE
:10148000E32E80E421C0C701B60120E03DE241E344
:1014900051E00E944C2EE901689760E073ED8EECFC
:1014A0009EEF0E94282E6C0D7D1D8E1D9F1D660FC8
:1014B000771F881F991F21E732E040E050E00E942B
:1014C0004C2EF22EE32E80E66C2F6F71680F85E7AD
:1014D0000E949F096E2D86E70E949F096F2D87E766
:1014E0000E949F09DF91CF91FF90EF90DF90CF9006
:1014F0000895682F8DE60E949F0908958F929F920C
:10150000AF92BF92CF92DF92EF92FF92CF93DF9391
:10151000D82F83E00E94990980936F0584E00E9490
:10152000990980936E0560E086E00E949F0961E062
:1015300087E00E949F096FE789E00E949F0965E0AC
:101540008AE00E949F0962E18BE00E949F0965E1A9
:101550008CE00E949F096DEF8DE00E949F0960E082
:101560008EE00E949F09DD2319F08BE291E008C014
:1015700020919B0533E1239FC0011124825C9E4F83
:101580000E94CC096CE880E30E949F096FE082E32F
:101590000E949F0962E483E30E949F0980919C0559
:1015A00087FF02C064E101C06AE084E30E949F09F2
:1015B0006AE285E30E949F096DE286E30E949F092B
:1015C00064ED87E30E949F0960E088E30E949F0921
:1015D00060E089E30E949F09D11109C0C0907D0598
:1015E000D0907E05E0907F05F090800507C0C5E9AA
:1015F000CC2EC1ECDC2EED2CCEEDFC2ECAE38F2CD4
:101600009924AA24BB24682D8C2F0E949F09682D41
:1016100085E08C0F0E949F09FE2CED2CDC2CCC2445
:10162000CF5FCE3361F76FEF83E40E949F096FEFC6
:1016300084E40E949F096FEF85E40E949F096FEF89
:1016400086E40E949F09DD2311F066E002C06091EC
:1016500081058DE60E949F0960E089E70E949F094D
:10166000609182058AE70E949F0960E083E70E94FB
:101670009F0960E084E70E949F09D11109C0609131
:10168000790570917A0580917B0590917C0504C065
:1016900060EC72E98DEE99E10E940E0ADF91CF9124
:1016A000FF90EF90DF90CF90BF90AF909F908F9082
:1016B000089561E087E00E949F0964E28EE70E943E
:1016C0009F0963E088E00E949F0960E088E00E9433
:1016D0009F0965E087E00E949F0962E085E00E9423
:1016E0009F0983E00E94990980936F0584E00E941E
:1016F000990980936E05089583E00E94990980936B
:101700006F0584E00E94990980936E0561E087E08F
:101710000E949F096AE070E080E090E00E94172933
:101720000E94590B00000895CF92DF92FF920F9311
:101730001F93CF93DF931F92CDB7DEB7082F162FDD
:101740008EE399830E949F09F02EC02E9981D92E95
:101750008C2D8F19811738F4F60161916F018FE795
:101760000E949F09F5CF64E085E00E949F0983E015
:101770000E94990980936F0584E00E9499098093E3
:101780006E050E94F42860936A0570936B05809340
:101790006C0590936D0569E087E00E949F0981E0E8
:1017A000809371050F90DF91CF911F910F91FF9062
:1017B000DF90CF9008950F931F930E94940B809118
:1017C0007105813099F40E94F42800916A05109106
:1017D0006B0520916C0530916D05601B710B820BC0
:1017E000930B603A76488140910548F380917105EA
:1017F000813031F46EE971E080EE95E00E94E02ADC
:101800001F910F9108950F931F938091710582305E
:1018100021F41092710581E020C080917105813022
:10182000D9F40E94F42800916A0510916B0520916B
:101830006C0530916D05601B710B820B930B613A47
:1018400076488140910540F061E087E00E949F0961
:101850001092710582E001C080E01F910F91089500
:10186000CF93DF93EC014AE050E06D2F70E080EE03
:1018700095E00E94AE2B6EE280EE95E00E94B22AC7
:10188000BE0184E0769567958A95E1F76F707727BA
:101890004AE050E080EE95E00E94AE2B6EE280EED2
:1018A00095E00E94B22ABE016F7077274AE050E0AF
:1018B00080EE95E00E94AE2BDF91CF910895D82F56
:1018C000C0E0CD1780F42D9A64E670E080E090E0EF
:1018D0000E9417292D9864E670E080E090E00E9455
:1018E0001729CF5FEECF6CE271E080E090E00E94BC
:1018F0001729E6CF0F931F93CF93DF93EC01062FA9
:1019000015E0115051F0CE010E94A930081741F0A6
:10191000602FCE010E94B130F4CF82E00E945F0CB4
:10192000DF91CF911F910F910895A0E0B0E0EBE916
:10193000FCE00C948F2E482E562EC0E0D0E0612C97
:10194000712CE12CF12C00E010E041100CC06090F3
:10195000D20586E4689E3001112459E1E52EF12C70
:1019600008EB15E01EC091E049120FC06090D2054F
:10197000E6E46E9E30011124FBE16F0E711C49E21A
:10198000E42EF12C04E715E00CC082E0481209C0F7
:1019900028E1622E77247394EE24E394F12C01ED78
:1019A00015E043018C0E9D1E109273051092720576
:1019B0003401A62CA818B12CC30101966C01AE14F9
:1019C000BF04A8F4A00EB11E511006C0C3010E94AE
:1019D000A930F501808305C0F5016081C3010E9433
:1019E0007A0CF50180810E9461063601E2CFC301C5
:1019F000511018C0C3010E94A930B82EC6010E9420
:101A0000A9302B2D30E0322F2227282B8091720510
:101A1000909173058217930779F4C0E0D0E05524C4
:101A2000539493CF3601609173050E947A0C6091B4
:101A30007205C6010E947A0CC05EDE4FC13E92E084
:101A4000D90708F482CF852DCDB7DEB7E0E10C943D
:101A5000AB2E61E082E00E94950C089560E082E088
:101A60000E94950C8091D105853020F01092D1050F
:101A70000E94290D8091D1058093D205089561E0DF
:101A800080E00E94950C61E081E00E94950C089531
:101A900060E080E00E94950C882351F060E081E0D6
:101AA0000E94950C882321F080917405883349F0B9
:101AB0000E94BF060E947A0681E00E94DF060E9413
:101AC0003F0D0895882319F06AEA71E002C06EEABA
:101AD00071E080EE95E00E94E02A0895FF920F9356
:101AE0001F93CF93DF9369EC7BE080EE95E00E943B
:101AF0008C2A4091790550917A0560917B0570910F
:101B00007C052AE030E080EE95E00E94B52B63EB87
:101B10007BE080EE95E00E948C2A40917D055091FB
:101B20007E0560917F057091800520E130E080EEB8
:101B300095E00E94B52B6DE97BE080EE95E00E9478
:101B40008C2A4AE050E06091810580EE95E00E9489
:101B5000DD2B67E87BE080EE95E00E948C2A4AE06E
:101B600050E06091820580EE95E00E94DD2B61E7F8
:101B70007BE080EE95E00E948C2AC3E8D5E0F12C52
:101B80008E0188818823A9F0FF2031F061EB71E09C
:101B900080EE95E00E94AF2A21964AE050E0F801DD
:101BA000608180EE95E00E94A62BF394F8E1FF128D
:101BB000E7CF80EE95E00E94BA2A6BE57BE080EEED
:101BC00095E00E948C2A4AE050E060919B0580EEEF
:101BD00095E00E94DD2B66E47BE080EE95E00E94BC
:101BE0008C2AE0919C05E770F0E0EE0FFF1FEE57A6
:101BF000FC4F6081718180EE95E00E94E02A61E3F4
:101C00007BE080EE95E00E948C2A80919C05887193
:101C1000883069F028F4811113C068E27BE00CC0C1
:101C2000803141F0883161F46CE07BE005C06CE10B
:101C30007BE002C066E17BE080EE95E00E94CE2A68
:101C400068EF7AE080EE95E00E948C2A409175055D
:101C50005091760560917705709178052AE030E023
:101C600080EE95E00E94B52B6FED7AE080EE95E076
:101C70000E948C2A8091BD0580710E94620D66ECE5
:101C80007AE080EE95E00E948C2A8091BD058074F8
:101C90000E94620D6DEA7AE080EE95E00E948C2A47
:101CA0008091BD0580720E94620D60E97AE080EE4D
:101CB00095E00E948C2A84E795E00E94F407AB012E
:101CC000BC012AE030E080EE95E00E94972B6BE8A3
:101CD0007AE080EE95E00E948C2A84E795E00E94ED
:101CE000F4079B01AC0160E472E48FE090E00E9495
:101CF0004C2EBA01A9012AE030E080EE95E00E9466
:101D0000972B68E87AE080EE95E00E94CE2ACDB766
:101D1000DEB7E5E00C94B62E8F929F92AF92BF9201
:101D2000CF92DF92EF92FF92811107C06FE77AE0C6
:101D300080EE95E00E94CE2A2FC090E00E947407AA
:101D400024E630E040E050E00E944C2ECA01B90188
:101D50002AE030E040E050E00E944C2E49015A0158
:101D60006B017C012AE030E0B501A40180EE95E032
:101D70000E94972B6EE280EE95E00E94B22A2AE044
:101D800030E0B701A60180EE95E00E94972B63E753
:101D900080EE95E00E94F22AFF90EF90DF90CF90C6
:101DA000BF90AF909F908F9008951F93CF93DF9334
:101DB00065E77AE080EE95E00E948C2A80919D058F
:101DC000813041F46CE57AE080EE95E00E94CE2A05
:101DD00010E050C0823019F465E47AE0F5CF843029
:101DE00019F461E37AE0F0CF853091F766E27AE0AA
:101DF000EBCFC12FD0E0C930D1050CF441C068E36E
:101E0000610F80EE95E00E94B22A6EE17AE080EEEA
:101E100095E00E948C2ABE016F5F7F4F4AE050E040
:101E200080EE95E00E94762B63E17AE080EE95E00B
:101E30000E948C2AC356DA4FE981E03218F566E039
:101E40007AE080EE95E00E948C2A8981803130F022
:101E50006DE673E080EE95E00E94AF2A69816F70B5
:101E600070E06F5F7F4F4AE050E080EE95E00E94A7
:101E70007F2B1F5F80914605181708F4BACF0FC05B
:101E800061E3BECFEF70F0E0EE0FFF1FEE56FC4FA8
:101E90006081718180EE95E00E94E02AEACF6BEECE
:101EA00079E080EE95E00E948C2A8091B5050E9431
:101EB0008C0E60ED79E080EE95E00E948C2A809196
:101EC000B6050E948C0E65EB79E080EE95E00E94ED
:101ED0008C2A8091B7050E948C0E6AE979E080EE29
:101EE00095E00E948C2A4091AD055091AE0560911D
:101EF000AF057091B005411551056105710539F1C6
:101F00002AE030E080EE95E00E94B52B67E679E0AC
:101F100080EE95E00E948C2A8091B1050E9499077D
:101F2000AB01BC012AE030E080EE95E00E94B52BC9
:101F300063E479E080EE95E00E948C2A4AE050E06C
:101F40006091B20580EE95E00E94DD2B06C06AE349
:101F500079E080EE95E00E94CE2A6DE179E080EE96
:101F600095E00E948C2A6091B3057091B4054AE017
:101F700050E080EE95E00E94C72B60E079E080EEB3
:101F800095E00E948C2A6091AC05603450F470E0BA
:101F90006F5F7F4F4AE050E080EE95E00E947F2B1C
:101FA00006C067EF78E080EE95E00E94CE2A6AEDE9
:101FB00078E080EE95E00E948C2A8091AB0580FF4E
:101FC00003C063EB71E002C067EB71E080EE95E067
:101FD0000E94E02A6DEB78E080EE95E00E948C2A6A
:101FE0008091AB0582700E94620D6EE978E080EE10
:101FF00095E00E948C2A8091AB0584700E94620D4E
:102000006FE778E080EE95E00E948C2A8091AB0526
:1020100088700E94620DDF91CF911F9108950F93F8
:102020001F93CF93DF93209143052F3FA9F56FEFC7
:1020300075E080EE95E00E948C2A83E893E00E9490
:10204000300C6EED75E080EE95E00E948C2A809158
:102050004405909145050E94300C6BEA75E080EED6
:1020600095E00E94CE2A68E875E080EE95E00E9437
:10207000CE2A60E775E080EE95E00E94CE2A6BE400
:1020800075E080EE95E00E94CE2A80EE95E00E94F9
:10209000BA2A0E94D50E68C012160CF065C033270C
:1020A00027FD30958091460590E0821793070CF448
:1020B0005BC066E375E080EE95E00E948C2A60913B
:1020C0004305772767FD70954AE050E080EE95E084
:1020D0000E947F2B6BE075E080EE95E00E948C2AD9
:1020E00010E008E2809147051817D0F5C12FD0E025
:1020F000CC0FDD1FC85BDA4F288130E080914305AB
:10210000992787FD909501972817390739F56BEBCB
:1021100071E080EE95E00E94AF2A4AE050E0602F27
:1021200080EE95E00E94A62B6FEB71E080EE95E0CB
:102130000E94AF2AE981EF70F0E0EE0FFF1FEE562C
:10214000FC4F6081718180EE95E00E94AF2A63ECC4
:1021500071E080EE95E00E94AF2A0F5F1F5FC2CF53
:1021600080EE95E00E94BA2ADF91CF911F910F91E6
:102170000895FF920F931F93CF93DF93C3E8D5E0A9
:10218000F12C8E0188818823D1F165EC71E080EE1D
:1021900095E00E94AF2A4AE050E06F2D80EE95E076
:1021A0000E94A62B62ED71E080EE95E00E94AF2ABE
:1021B0002196F801208130E0A0E1B7E20E94062ECE
:1021C0009B01AC01A0918205B0E00E94152EAB01ED
:1021D000BC018091790590917A05A0917B05B09121
:1021E0007C05480F591F6A1F7B1F2AE030E080EEF4
:1021F00095E00E94B52BF394F8E1FF12C2CFCDB762
:10220000DEB7E5E00C94B62E1092DD0485E6EEED27
:10221000F4E0DF011D928A95E9F70895CF93C82F66
:102220008F3719F0883009F045C0E091DD04EE23C6
:10223000D9F1E150E093DD04F0E0E252FB4F10826F
:102240006DE070E080EE95E00E945906C0E080915C
:10225000DD04C81760F4EC2FF0E0E252FB4F608120
:1022600070E080EE95E00E945906CF5FF0CF60E20B
:1022700070E080EE95E00E9459066DE070E080EE1F
:1022800095E00E945906C0E08091DD04C81778F5FA
:10229000EC2FF0E0E252FB4F608170E080EE95E0C1
:1022A0000E945906CF5FF0CF67E080EE95E00E9474
:1022B000B22A1DC08B3119F40E9404111AC08D304E
:1022C000C1F08A30B1F08091DD04843668F76C2F5C
:1022D00070E080EE95E00E945906E091DD0481E017
:1022E0008E0F8093DD04F0E0E252FB4FC08380E06C
:1022F00001C081E0CF910895CF93C82F0E94F428A8
:102300006093C6047093C7048093C8049093C90473
:10231000C093DB04CC2329F040E051EE60E070E094
:1023200004C040E855E260E070E080EE95E00E9475
:102330003C2DCF9108959091CA04492F4F7050E0E1
:10234000BA016F5F7F4F292F30E0E4E03595279584
:10235000EA95E1F76217730759F0FA01E553FB4F6D
:10236000808381E0890F8F70907F892B8093CA04CE
:1023700008956EE770E080EE95E00E94590608959A
:10238000A3E1B1E0E6ECF1E10C94902EE3E8F5E096
:10239000712C8191882321F0739428E17212F9CF76
:1023A00066ED71E080EE95E00E94E02A4AE050E0A0
:1023B000672D80EE95E00E94DD2B80E00E947E0A72
:1023C0000E94590B8E010E5F1F4FC12CD12C76013C
:1023D000C39466246A945C2C0E94E8284B015C013B
:1023E0002091820530E0A0E1B7E20E94062E9B0119
:1023F000AC01C701B6010E94282E209179053091C9
:102400007A0540917B0550917C05620F731F841FF4
:10241000951F2091B9053091BA054091BB055091A7
:10242000BC05261737074807590718F4F8016082DA
:1024300025C08C2D0E94B20961E070E080E090E040
:102440000E941729F80110820E94E828681979096A
:102450008A099B09643F71408105910540F40E94FF
:10246000C809F8019081981778F78083EDCF50FE66
:1024700003C02C982D9A02C02C9A2D982FEFC21AC7
:10248000D20AE20AF20A0F5F1F4F8FEFC816D1047B
:10249000E104F10409F09FCFCE019395FC01D82E01
:1024A0007FEF68EC2E2F281B271510F051E056C047
:1024B000DE01129651E02FEF41E03D91321710F00E
:1024C000322F01C0452F5F5F5F3F11F0232FF5CF03
:1024D0004193242F30E0A1E0B0E0AC0FBD1FA20F6C
:1024E000B31F5C93413079F0DE01A20FB31F5C9300
:1024F000423049F0AFEFBFEFAC0FBD1FA20FB31FCB
:102500006C934E3F78F6A2E0B0E0AC0FBD1FA20F77
:10251000B31F7C934D3F30F6A3E0B0E0AC0FBD1F7E
:10252000A20FB31F6C93BECF452F242F30E0FC01C8
:10253000E20FF31F6081AFEFB0E0AC0FBD1FA20F41
:10254000B31F2C91621748F44150DC01A40FB11D58
:102550002C9120836C934111E8CF5F5F571520F3D6
:10256000372D369520E0231770F4DC01A20FB11D42
:102570004C91522F530FFC01E50FF11D50815C93DC
:1025800040832E5FF0CFF3E8EF2EF5E0FF2E8C01B5
:10259000802F8D19871598F4F801C1908F014AE0BA
:1025A00050E06C2D80EE95E00E94A62B6CE280EE50
:1025B00095E00E94B22AF701C1927F01E9CF80EE37
:1025C00095E00E94BA2A81E0CD5EDE4FEFE00C94E8
:1025D000AC2E1F920F920FB60F9211240F931F93E0
:1025E0002F933F934F935F936F937F938F939F931B
:1025F000AF93BF93EF93FF934091BD055091BE05FC
:102600006091BF057091C00589B18A019B0100747A
:1026100011272227332783FB882780F990E0A0E049
:10262000B0E0081719072A073B0709F468C0809132
:102630008400909185001092850010928400209172
:10264000A70421115CC045FD02C096958795853C85
:1026500029E09207C0F180910A0190E0A0E0B0E08B
:102660000CE176956795579547950A95D1F74115F1
:1026700051056105710521F441E050E060E070E032
:10268000481759076A077B07D8F480910A018F3FE2
:10269000B9F040E080910A01481780F4842F90E05F
:1026A000880F991FFC01E957FB4F20813181FC0104
:1026B000E55FFE4F318320834F5FECCF1092A8047B
:1026C00010920A011CC08D3B22E09207A8F02091D5
:1026D0000A01203188F410910A0121E0210F209392
:1026E0000A010E94DE08E12FF0E0EE0FFF1FE9571C
:1026F000FB4F9183808303C08FEF80930A01FF918A
:10270000EF91BF91AF919F918F917F916F915F9169
:102710004F913F912F911F910F910F900FBE0F90EE
:102720001F90189583E0809380008AE18093810058
:102730008FEF9FEF909389008093880010926F0035
:1027400088E080936D00E8E6F0E08081846080831B
:102750000895CF93DF930E942E0D8091D20584308F
:1027600039F585E00E940D2AC1E0D0E0892B11F4F3
:10277000C0E0D0E086E00E940D2A892B19F082E0AB
:1027800090E002C080E090E08C2B9D2B8230910580
:1027900039F08330910539F0019739F481E006C0B2
:1027A0001092D20505C082E001C083E08093D2057B
:1027B000DF91CF9108956F3018F086958058089575
:1027C00089E0689F802D11240895A0E0B0E0EBEE31
:1027D000F3E10C94972EC82F0E94F428009138043E
:1027E0001091390420913A0430913B046B017C0133
:1027F000C01AD10AE20AF30A9701860149E8C41611
:1028000043E1D406E104F10410F010923C0460931B
:1028100038047093390480933A0490933B042091D8
:10282000A7048FEF820F8230D8F5E0913C04EE23AD
:1028300009F44EC1E13011F482E0B8C1E03108F092
:1028400034C181E08E0F80933C04F0E0E957FB4FE8
:10285000C083803109F0ACC1E9E8F4E0213029F40B
:10286000A181A695A695808108C080819181A92F1C
:10287000A695A695A69596958795A03148F4B0E0C3
:1028800090E0AA0FBB1FA55FBE4F11969C938E933D
:102890001092A804329684E0E739F807F9F688C167
:1028A000233009F005C1E0913C04E11104C0CF30B0
:1028B00009F07EC10DC1E83148F481E08E0F8093AC
:1028C0003C04F0E0EA57FB4FC08372C1E83109F0E5
:1028D000ECC0C111EAC040E050E0ABE0CA01B3E097
:1028E000880F991FBA95E1F7A49F9001A59F300D1D
:1028F0001124F901E957FB4F6081E1817E2F777048
:1029000075956795FC01EE0FFF1FE55FFE4F718324
:102910006083F901E857FB4FB081B695B695B6953F
:10292000E181FE2FF295FF0FF07E6F2F6B2BE69566
:10293000E695E6957E2F777075956795FC01EE0F0D
:10294000FF1FE35FFE4F71836083F901E757FB4F81
:10295000B081B295B695B695B370C181DC2FDD0F0D
:10296000DD0F6D2F6B2BC295C695C695C370E281A6
:10297000E170EE0FEE0F7E2F7C2B75956795FC01B5
:10298000EE0FFF1FE15FFE4F71836083F901E55792
:10299000FB4FB081B695E181FE2FF795FF27F795A4
:1029A0006F2F6B2BE6957E2F777075956795FC01E1
:1029B000EE0FFF1FEF5EFE4F71836083F901E45756
:1029C000FB4FB081B295BF70E181FE2FF295F07F91
:1029D0006F2F6B2BE295EF707E2F77707595679553
:1029E000FC01EE0FFF1FED5EFE4F71836083F90166
:1029F000E357FB4FB081BB1FBB27BB1FC181DC2F3F
:102A0000DD0F6D2F6B2BCC1FCC27CC1FE281E37029
:102A1000EE0F7E2F7C2B75956795FC01EE0FFF1F47
:102A2000EB5EFE4F71836083F901E157FB4FB0818C
:102A3000B695B695E181FE2FF295FF0FFF0FF07C62
:102A40006F2F6B2BE695E6957E2F777075956795C2
:102A5000FC01EE0FFF1FE95EFE4F71836083F901F9
:102A6000E057FB4F20812295269527703181E32F77
:102A7000EE0FEE0FEE0F6E2F622B732F7295769581
:102A8000777075956795FC01EE0FFF1FE75EFE4FAF
:102A9000718360834F5F5F4F4230510509F01ECF55
:102AA00080919D0483FF1092A80410923C0480C082
:102AB000243009F07DC060913C0461110BC0C83A1C
:102AC000B1F4109273051092720588EA0E946106B3
:102AD00081E06CC0613019F4C093370404C06230E7
:102AE00031F4C09336048C2F0E9461065AC0E091E5
:102AF00036042E2F30E0220F331F462F50E0C9013D
:102B00000296841795073CF0633268F7FA01EC5798
:102B1000FB4FC083E8CF2D5F3F4F8C2F90E060913B
:102B20007205709173054217530749F4982F88274F
:102B300086279727909373058093720532C0681794
:102B4000790769F580913704813049F5E13118F052
:102B500080E180933604F0903604C8E8D4E000E0C9
:102B600010E00F15D0F4FE013197808190E0982F8E
:102B700088272881822B43E0969587954A95E1F72F
:102B80000E94DE08F801EE0FFF1FE55FFE4F918304
:102B900080830F5F1F4F2296E4CF1092A8041092FB
:102BA0003C0480913C04882319F08F5F80933C049F
:102BB000CDB7DEB7E8E00C94B32ECF93DF93E82FC8
:102BC000F0E0E854FA4FE185E03150F4F894F0E099
:102BD000EE0FFF1FE55FFE4F80819181789437C033
:102BE000E13131F0E23141F0E03161F582E101C0E3
:102BF00083E10E94362A2BC085E00E940D2AC1E0A5
:102C0000D0E0892B11F4C0E0D0E086E00E940D2ACC
:102C1000892B19F082E090E002C080E090E08C2BDC
:102C20009D2B8230910541F08330910541F0019751
:102C300061F086EA92E00BC08CE090E008C089E584
:102C400091E005C080E092E002C084EF93E0DF9164
:102C5000CF910895A2E2B0E0E0E3F6E10C948D2E6E
:102C60009E012F5F3F4F80E1D9011D928A95E9F7C0
:102C700064E072E080EE95E029A33AA30E94E02A86
:102C80000E947C0B1D8A1E8A1F8A188E312C212CD3
:102C900000E0812C912C540170E4472E71EE572EE8
:102CA0007DE9672E78E1772EE0E5CE2EE3ECDE2E8F
:102CB000E12CF12C84EF91E0A0E0B0E08D8F9E8FAD
:102CC000AF8FB8A380EC91EDA8E9BBE1898F9A8F13
:102CD000AB8FBC8F80E491EEADE9B8E1898B9A8B24
:102CE000AB8BBC8B80EE95E00E94F42B892B09F412
:102CF000E1C080EE95E00E94212C9C0133272C320C
:102D0000310509F442C0ACF42332310509F0ABC0FF
:102D100019821A821B821C821D821E821F821886C3
:102D200019861A861B861C861D861E861F86188A93
:102D300060C02434310529F02335310509F4B2C0CF
:102D400092C064E480EE95E00E94B22A2AE030E06E
:102D500040E451EE6DE978E180EE95E00E94402B71
:102D60006CE280EE95E00E94B22A2AE030E040EC6E
:102D700051ED68E97BE180EE95E00E94402B6CE22A
:102D800080EE95E00E94F22AADCF0F5F043009F08B
:102D9000A9CF29813A814B815C81A8EEB3E00E94E2
:102DA000152E698B7A8B8B8B9C8B2D813E814F816D
:102DB00058850E94152E698F7A8F8B8F9C8F29855D
:102DC0003A854B855C852D8F3E8F4F8F58A32D857F
:102DD0003E854F8558890E94152E6B017C0160321B
:102DE0003EE473078105910530F462E38CE10E94B3
:102DF0009F0900E077CF603345E7740781059105AF
:102E000010F462E2F3CF60345CE975078105910547
:102E100010F466E2EBCF80E5C81683ECD806E10437
:102E2000F10410F462E1E2CF90E6C9169AEED906F9
:102E3000E104F10410F465E1D9CFA0E7CA16A1E1DD
:102E4000DA06A1E0EA06F10410F461E0CFCFB0EABF
:102E5000CB16B6E8DB06B1E0EB06F10410F463E054
:102E6000C5CF65E0C3CF10ED180F1A3008F03ACF88
:102E7000E1E0F0E0EC0FFD1F24E0029FE00DF11D0A
:102E800011242081318142815381AAE0B0E00E9467
:102E9000152E610F711D811D911D608371838283C9
:102EA000938320CF49885A886B887C88812C912C09
:102EB000540118CF81149104A104B10489F4C30111
:102EC000B2010E940E0A61E070E080E090E00E9492
:102ED00017291D8A1E8A1F8A188E312C22242A94B3
:102EE0008D8D9E8DAF8DB8A188169906AA06BB065A
:102EF000D0F40E94C8092D893E894F89588D280F2A
:102F0000311D411D511D2D8B3E8B4F8B588F381617
:102F100008F4382E821508F4282E3FEF831A930AFE
:102F2000A30AB30A56C0C301B20128EE33E040E061
:102F300050E00E944C2EBA01A9012AE030E080EE58
:102F400095E00E94972B6CE280EE95E00E94B22AF9
:102F50004AE050E0632D80EE95E00E94A62B6CE2E3
:102F600080EE95E00E94B22A6D897E898F89988DC6
:102F7000A50194010E944C2EBA01A9012AE030E07B
:102F800080EE95E00E94972B6CE280EE95E00E9427
:102F9000B22A4AE050E0622D80EE95E00E94A62B16
:102FA0006CE280EE95E00E94F22A4C0C5D1C6E1CD7
:102FB0007F1C898D9A8DAB8DBC8D84159505A605DA
:102FC000B70520F449885A886B887C88812C912C1D
:102FD000540129893A894B895C89283E334041054F
:102FE000510509F07FCEA296E2E10C94A92EACE146
:102FF000B0E0EDEFF7E10C94972E0E94F4286B01FE
:103000007C0181E00E947E0A14E703E0198361E0FD
:10301000CE0101960E94DB0B009371050E94590BB3
:103020006AEF70E080E090E00E94172980917105BE
:10303000833089F480EE95E00E94F42B892B59F4BB
:103040000E94F4286C197D098E099F096038734C21
:10305000894C9140D8F280917105833009F44FC0BA
:103060008FE70E9477090E948A098983843511F0CD
:1030700083E05CC00E948A09109244058093450554
:103080000E948A092091440530914505280F311D81
:1030900030934505209344050E948A098093460594
:1030A0000E948A0980934705813110F7F12C0F2D7A
:1030B00010E08091470590E0880F991F08171907C5
:1030C00040F40E948A09F801E85BFA4F8083F39488
:1030D000EECF80E7898361E0CE0101960E94DB0B91
:1030E00083E0809371050E94590B62E370E080E0F9
:1030F00090E00E94172980917105833011F482E0DD
:1031000015C08FE70E9477090E948A09898380355C
:1031100009F0AECF0DE915E00E948A09F80181930C
:103120008F01F5E0083B1F07B9F781E06C96E8E0F6
:103130000C94B32E80914305992787FD9095A92F74
:10314000B92FFC013196EB30F10508F066C0EC5C5C
:10315000FF4F0C94C42E62E778E080EE95E00E9469
:10316000CE2A83E893E00E94300C6AE578E080EE96
:1031700095E00E94CE2A65E378E080EE95E00E941B
:10318000CE2A6BE078E080EE95E00E94CE2A6AEECF
:1031900077E080EE95E00E94CE2A6DEB77E080EE3E
:1031A00095E00E94CE2A67E977E080EE95E00E94E4
:1031B000CE2A63E777E080EE95E00E94CE2A6CE4A9
:1031C00077E080EE95E00E94CE2A80EE95E00E94A6
:1031D000BA2A0E946E0D21C06FE277E01AC06AE041
:1031E00077E017C065EF76E014C066ED76E011C0B9
:1031F00062E976E00EC06DE776E00BC068E676E047
:1032000080EE95E00E94CE2A62E276E002C06CE099
:1032100076E080EE95E00E94CE2A6AE070E080E0E1
:1032200090E00E94172980EE95E00E94F42B892BF4
:1032300029F080EE95E00E94212CF5CF0895ACE1B5
:10324000B0E0E5E2F9E10C94972E909143059F3FA1
:1032500009F023C1482F50E0FA013A97EF36F10503
:1032600008F00FC1E15CFF4F0C94C42E61E172E0E5
:10327000A0C06DE172E080EE95E00E94E02A85E753
:1032800089838BE1EDE9F5E0DE01129601900D9264
:103290008A95E1F76CE1CE0101960E94DB0B0E945A
:1032A000590B83E08093710568EC70E080E090E05A
:1032B0000E94172980917105843009F0E2C08FE7E0
:1032C0000E9477090E948A098983853509F0D9C04F
:1032D0006DEE74E080EE95E00E94CE2A6FEC74E013
:1032E00080EE95E00E94CE2A61EB74E096C065E323
:1032F00072E080EE95E00E94E02A89E6898361E031
:10330000CE0101960E94DB0B0E94590B83E0809353
:10331000710568EC70E080E090E00E9417298091D0
:103320007105843009F0ADC08FE70E9477090E94D3
:103330008A0989838E010E5F1F4F7E014DE1E40EE5
:10334000F11C0E948A09F80181938F01EE15FF0597
:10335000C1F78BE1FE013296ADE9B5E001900D9227
:103360008A95E1F78981893409F08BC063E974E0BB
:1033700080EE95E00E94CE2A65E774E080EE95E04D
:103380000E94CE2A67E574E048C06FE472E080EEE8
:1033900095E00E94E02A8EEF8093430572C0805230
:1033A0008750805390914605981708F066C06EE5E7
:1033B00072E080EE95E00E94E02A63C084E1809391
:1033C000430560E274E029C085E18093430569EE1E
:1033D00073E023C086E18093430562EB73E01DC078
:1033E00087E18093430568E673E017C088E1809326
:1033F000430567E573E011C089E18093430563E409
:1034000073E00BC08AE1809343056EE273E005C070
:103410008BE18093430566E073E080EE95E00E94C7
:10342000CE2A2FC06CEE72E080EE95E00E94CE2A8C
:103430008091AB0591E01DC066ED72E080EE95E0F5
:103440000E94CE2A8091AB0592E013C061EC72E03D
:1034500080EE95E00E94CE2A8091AB0594E009C0F1
:1034600066EA72E080EE95E00E94CE2A8091AB057C
:1034700098E089278093AB058FEF809343050E94E6
:103480000F1080EE95E00E94F42B892B09F45BC1AC
:1034900080EE95E00E94212CF4CF0E940E1188232B
:1034A00009F451C18091DD04811104C08FEF809334
:1034B000430541C140E050E060E070E08EED94E0F3
:1034C0000E943B2F40914305042F112707FD1095C3
:1034D000212F312FF8013197EB31F10508F01BC195
:1034E000E255FF4F0C94C42E552747FD509520916F
:1034F000460530E0241735070CF40DC18B019C0103
:103500000150110921093109003211052105310548
:1035100058F0C0904705E9E4F5E0F12CD12CA8E281
:10352000EA2E415051090FC0FA01E356FA4F61509B
:103530006083D9C0DF0111972C9130E02417350743
:1035400029F0F3943296FC10F5CFCBC00E2D10E08D
:1035500020E030E0061717072807390741F42081DB
:10356000DA01A356BA4F11962C93DD24D394E39439
:10357000E8CF6F3F71058105910511F008F0CBC0D0
:103580006093B505B0C06F3F71058105910511F0DD
:1035900008F0C1C06093B605A6C06F3F71058105F4
:1035A000910511F008F0B7C06093B7059CC0209159
:1035B000DE0420622037E9F440E050E060E070E093
:1035C0008FED94E00E943B2F9B01AC01DC01CB010D
:1035D0000197A109B1090897A105B10508F0AEC08E
:1035E000A4EDB0E30E94152E6A5E7C4A8A46954E91
:1035F00024C02636E9F440E050E060E070E08FED52
:1036000094E00E943B2F9B01AC01DC01CB010197B0
:10361000A109B1090797A105B10508F08FC0A8EA73
:10362000B1E60E94152E645E7C438E46944E05C022
:10363000611571058105910579F08B019C0100549C
:10364000114E2D4938410138F0EF1F07FAEF2F07CF
:10365000F2E03F0708F05FC06093AD057093AE05E0
:103660008093AF059093B0053EC06F3F7105810513
:10367000910511F008F04FC06093B10534C08B0183
:103680009C0101501109210931090F3F1105210544
:10369000310508F040C06093B20525C08B019C0144
:1036A000045C1940210931090D344DE1140721054D
:1036B000310528F47093B4056093B30514C0611507
:1036C00071058105910521F48FEF8093AC050BC046
:1036D0006134710581059105F0F461506093AC058A
:1036E00002C0DD20C1F08091DC0481111AC08091FC
:1036F0007D0590917E05A0917F05B0918005019692
:10370000A11DB11D80937D0590937E05A0937F053B
:10371000B093800506C060E772E080EE95E00E94FD
:10372000E02A0E9404118FEF809343056AE080EE47
:1037300095E00E94F22A0E940F1005C061E070E03F
:1037400080E090E07ACF6C96E8E00C94B32E6AE5C6
:1037500072E080EE95E00E94CE2A62E472E080EE94
:1037600095E00E94CE2A80EE95E00E94F42B892BF2
:1037700031F080EE95E00E94212C0E941F190E94DA
:10378000F717823029F0833051F46DE072E002C007
:1037900064E272E080EE95E00E94CE2A08958FEFF9
:1037A000809343051092DC040E940F108091430522
:1037B0008E3F69F080EE95E00E94F42B892BB1F3E7
:1037C00080EE95E00E94212C0E941F19EFCF0895F2
:1037D0000F931F93109143051F3F09F0D2C0893406
:1037E00009F457C000F5883309F469C058F48033F0
:1037F00009F477C008F061C08B3109F440C0813210
:10380000B1F1B9C0813409F487C030F4893309F4C7
:1038100066C0803461F1AFC0823409F48EC0863452
:1038200009F448C0A8C0823609F487C078F4883506
:1038300031F128F48235C1F18335E1F09CC08A353D
:1038400009F494C0813609F467C095C0823761F1EC
:1038500028F4863679F18936E1F08DC0883779F021
:103860008A3709F483C0833709F085C003C061E15A
:1038700072E015C00E943F0D6EE872E004C00E9425
:10388000480D68EA72E080EE95E00E94E02A8EEF33
:1038900070C00E947A060E94BF0667EC72E080EE5C
:1038A00095E00E94E02A67C081E00E94DF0660EE9A
:1038B00072E0F5CF0E94B9105EC080535AC06AEF23
:1038C00071E080EE95E00E94CE2A90919C0588E000
:1038D000890F8871977E892B80939C051AC089E097
:1038E00048C067EE71E080EE95E00E94CE2A80919C
:1038F000BD059091BE05A091BF05B091C00520E126
:1039000082278093BD059093BE05A093BF05B09319
:10391000C005109343052FC061ED71E080EE95E086
:103920000E94CE2A8091BD059091BE05A091BF0551
:10393000B091C00540E4842710C060EC71E080EED7
:1039400095E00E94CE2A8091BD059091BE05A09180
:10395000BF05B091C00520E282278093BD059093FA
:10396000BE05A093BF05B093C00502C00E94A71B6F
:103970008FEF80934305809143058E3F09F0D4C0BB
:10398000DDC00E940E11882309F4D8C08091DD04A7
:10399000811104C08FEF80934305C6C040E050E022
:1039A00060E070E08EED94E00E943B2F00914305B3
:1039B000112707FD1095212F312FF8013197E9309C
:1039C000F10508F0B4C0E753FF4F0C94C42E8B01EF
:1039D0009C010154114E2D4938410F37104F2A4F89
:1039E000324008F0A4C06093790570937A05809303
:1039F0007B0590937C0577C060937D0570937E0571
:103A000080937F059093800581E08093DC046BC0F8
:103A1000683071058105910508F089C060938105C2
:103A200062C08B019C0101501109210931090A3042
:103A300011052105310508F07AC06093820553C055
:103A400061EB71E08EED94E00E94753010E000971C
:103A500099F00E944F30009779F0183130F4E12F3F
:103A6000F0E0EC58FA4F87871F5F61EB71E080E070
:103A700090E00E947530EBCF1831A8F5E12FF0E00F
:103A8000EC58FA4F17861F5FF7CF65307105810537
:103A9000910508F04CC060939B0525C08B019C01EB
:103AA000015011092109310906301105210531059F
:103AB000F0F520919C05287F262B20939C0513C0B0
:103AC0008B019C0101501109210931090115124C8A
:103AD0002140310560F560937505709376058093FC
:103AE0007705909378058091DC04811113C0809153
:103AF0007D0590917E05A0917F05B091800501968E
:103B0000A11DB11D80937D0590937E05A0937F0537
:103B1000B09380050E9404118FEF809343056AE003
:103B200080EE95E00E94F22A0E949A1807C060E792
:103B300072E080EE95E00E94E02AECCF1F910F9199
:103B400008958FEF809343051092DC040E949A1829
:103B5000809143058E3F69F080EE95E00E94F42B42
:103B6000892BB1F380EE95E00E94212C0E94E81B86
:103B7000EFCF6AE070E080E090E00E94172980EECD
:103B800095E00E94F42B892B29F080EE95E00E94AD
:103B9000212CF5CF0895CF93C82F682F80EE95E0A4
:103BA0000E944E2C909168059C2790936805CF91B8
:103BB0000895A1E0B0E0EFEDFDE10C949D2E998316
:103BC0000E94CB1D9981892F0E94CB1D2196E2E096
:103BD0000C94B92E1F93CF93DF93182FEB01109203
:103BE000680565EB70E080EE95E00E94590662E69C
:103BF00070E080EE95E00E945906812F0E94CB1D57
:103C0000CE010E94D91DDF91CF911F91089560913F
:103C1000680580EE95E00E944E2C0895A1E2B0E088
:103C2000E4E1FEE10C94992E7B018A018C3009F4C9
:103C300052C108F040C0863009F4BCC018F583308A
:103C400009F491C070F4813009F472C0823009F037
:103C500047C26BE170E082E00E94EA1D0DE915E0C9
:103C600078C0843009F487C0853009F039C260918A
:103C7000470570E0660F771F85E00E94EA1D08E4A3
:103C800015E086C0893009F4A7C070F4873009F4C4
:103C90009BC0883009F024C261E070E088E00E9497
:103CA000EA1D8091D20522C28A3009F4CAC08B3045
:103CB00009F4F1C015C28A3609F474C1D8F4873604
:103CC00009F439C138F4853609F40DC1863609F492
:103CD0001EC106C2883609F436C1893609F000C211
:103CE00061E070E089E60E94EA1D0E947A060E9467
:103CF000BF06F4C18D3609F4D3C138F48B3609F40C
:103D000090C18C3609F499C1EBC18E3609F4DBC140
:103D1000873C09F0E5C161E070E087EC0E94EA1D94
:103D200081E00E94CB1D0E94071E10926905E2C12E
:103D300069E270E081E00E94EA1D04E715E0F80105
:103D400081918F010E94CB1DF5E00D391F07B9F756
:103D5000CFC1F80181918F010E94CB1DF5E0083B96
:103D60001F07B9F7C5C161E070E083E00E94EA1D5A
:103D70000E94F717BBC161E070E084E00E94EA1D79
:103D800081E00E94CB1D0E94071E0E942A16B2C12C
:103D90008091470590E0880F991F9801285435407D
:103DA0002817390708F0A4C1F80181918F010E94FA
:103DB000CB1DEECF62E070E086E00E94EA1D83E852
:103DC00093E00E94D91D94C161E070E087E00E94F9
:103DD000EA1D809146058AC186E6898361E0CE01AD
:103DE00001960E94DB0B0E94590B83E080937105C2
:103DF00068EC70E080E090E00E94172980917105E6
:103E00008430D9F48FE70E9477090E948A09898358
:103E1000863469F460E270E089E00E94EA1D10E2F5
:103E20000E948A090E94CB1D1150D1F761C161E047
:103E300070E089E00E94EA1D51C161E070E089E014
:103E400052C169E170E08AE00E94EA1D1092B80553
:103E5000209170058091BD059091BE05A091BF0590
:103E6000B091C005222311F0806801C08F77809344
:103E7000BD059093BE05A093BF05B093C00508EBA8
:103E800015E0F80181918F010E94CB1DF5E0013D05
:103E90001F07B9F72DC161E270E08BE00E94EA1DB7
:103EA0008091A8048F3F39F08091A80491E0980F89
:103EB0009093A80402C08091A8040E94CB1D10E03A
:103EC000812F0E94DD150E9409090E94D91D1F5FE4
:103ED0001031B1F70DC161E070E08CE00E94EA1D85
:103EE0008091D10503C161E070E085E60E94EA1D82
:103EF00089E2E816F10409F0F8C0D801E4E7F5E03A
:103F00008D91819385E0ED39F807D1F7E7C061E045
:103F100070E086E60E94EA1DEBE1EE16F10409F07E
:103F2000E4C0D801EDE9F5E08D91819385E0E83BAF
:103F3000F807D1F7D3C061E070E087E60E94EA1D80
:103F40000E943F0DCBC061E070E088E60E94EA1D50
:103F500085E789838BE1EDE9F5E0DE0112960190BA
:103F60000D928A95E1F76CE1CE0101960E94DB0B80
:103F70000E94590B83E08093710560E273E080E05A
:103F800090E00E94172980917105843009F0ADC03E
:103F90008FE70E9477090E948A098983853509F095
:103FA000A4C09CC061E070E08AE60E94EA1D89E638
:103FB000898361E0CE0101960E94DB0B0E94590BC0
:103FC00083E08093710560E273E080E090E00E94FE
:103FD000172980917105843009F087C08FE70E940E
:103FE00077090E948A0989838E010E5F1F4F7E0127
:103FF000EDE1EE0EF11C0E948A09F80181938F0118
:10400000EE15FF05C1F78BE1FE013296ADE9B5E093
:1040100001900D928A95E1F78981893409F065C094
:104020005DC061E070E08BE60E94EA1DF8018081CE
:104030008093D2050E94480D51C061E070E08CE68B
:104040000E94EA1DF0E2EF16F10461F487E689832D
:1040500080E2F801DE01129601900D928A95E1F757
:1040600061E203C087E4898361E0CE0101960E948A
:10407000DB0B0E94590B83E0809371056CE474E0C4
:1040800080E090E00E94172980917105843069F5E5
:104090008FE70E9477090E948A09873431F51EC094
:1040A00061E070E08DE60E94EA1D89E1E816F10406
:1040B000E1F4D801E8EBF5E08D91819385E0E13DF5
:1040C000F807D1F70BC061E070E08EE60E94EA1DB0
:1040D000F80180818093D1050E94290D81E006C0FE
:1040E00061E070E08AEC0E94EA1D80E00E94CB1D36
:1040F0000E94071EA196E6E00C94B52EA0E0B0E069
:10410000E4E8F0E20C94972ECAECD3E014E606E063
:1041100035E0F32E44E0E42E53E0D52E62E0C62EC7
:1041200080EE95E00E94F42B892B09F49BC080EE71
:1041300095E00E94212C282F80933504409134046F
:1041400050E04730510560F7FA01EE52FF4F0C94F2
:10415000C42E853B29F781E080933404E1CF823679
:1041600009F07DC0C0923404DBCF80933304809388
:104170003204D0923404D4CF9C01332730933104DD
:104180002093300490913204982790933204E09267
:104190003404C6CF382F2227409130045091310487
:1041A000242B352B3093310420933004909132042A
:1041B000982790933204F09234042536310508F4A0
:1041C000AFCF61E070E08CEC0E94EA1D81E00E94BC
:1041D000CB1D0E94071E43C020912E0430912F0456
:1041E000F901E653FC4F8083909132049827909315
:1041F0003204C901019690932F0480932E042091DC
:104200003004309131048217930708F489CF00936A
:10421000340486CF8091320482130BC060912E0447
:1042200070912F044AEC53E0809133040E940E1EDB
:104230000DC062E070E08BEC0E94EA1D80913304B7
:104240000E94CB1D809168050E94CB1DFE01812F2D
:1042500011928A95E9F710922F0410922E04109271
:1042600034045ECFCDB7DEB7E8E00C94B32E81E026
:104270008093690580916905882349F080EE95E077
:104280000E94F42B892BB1F30E947E20F3CF089576
:10429000AAE2B0E0EEE4F1E20C94952E0E94E82848
:1042A0006B017C0181E00E947E0A80EE95E00E9415
:1042B000F42B892B29F080EE95E00E94212CF5CF7C
:1042C0002D9811E072E6B72EE9E2AE2E03E00E94CF
:1042D000E8286C197D098E099F09693C71058105E3
:1042E0009105D0F11123C1F10E94E8286B017C01F6
:1042F0002C9A80ED97E00E94A807B982E4E7F5E0E8
:10430000DE0112968A2D01900D928A95E1F76AE2FC
:10431000CE0101960E94DB0B2C9880E090E00E9479
:10432000A807009371050E94590B62E370E080E0DA
:1043300090E00E94172980917105843061F4009308
:1043400071058FE70E9477090E948A0911E0823483
:1043500019F410E001C011E08BE00E940D2A892BB6
:1043600081F411E00EC02D9A2C9A80EE95E00E9407
:10437000212C8D309105A9F05CF40A9791F02D98CD
:104380002C9880EE95E00E94F42B892B61F79FCF4B
:104390008332910579F08234910589F70E943721A3
:1043A000EECF62EB71E080EE95E00E94CE2A0E9493
:1043B000A11DE5CF0E942A16E2CF8F929F92AF9265
:1043C000BF92CF92DF92EF92FF921F93CF93DF9332
:1043D0008BE00E940D2A892B09F089C068EC70E0FF
:1043E00080E090E00E94172980E090E00E94A807FA
:1043F0000E94E8284B015C016B017C0180ECC80E37
:1044000082E1D81EE11CF11C0E94E8286C157D0594
:104410008E059F0530F48BE00E940D2A892BA1F3B5
:1044200064C08BE00E940D2A892B09F05EC080EDEC
:1044300097E00E94A8070E94E8286B017C01D0E069
:10444000C1E088E4880E86E2981EA11CB11C11E030
:104450008BE00E940D2A892B21F58C149D04AE045B
:10446000BF0430F480ED97E00E94A807D1E0F0CFC0
:104470000E94E8286C197D098E099F09693C710525
:104480008105910528F30E94E8286B017C01C12772
:1044900019F080ED97E002C080E090E00E94A8074C
:1044A000D7CF80E090E00E94A807DD23B9F080918B
:1044B000D10590E0019665E070E00E94382E80936F
:1044C000D1050E94290D0E94A9130E94480D64EF96
:1044D00071E080E090E00E94172909C080E00E940E
:1044E000DF060E94C0110E943F0D0E944821DF910B
:1044F000CF911F91FF90EF90DF90CF90BF90AF9042
:104500009F908F900895CF92DF92EF92FF9280E07C
:104510000E94DA070E94B10761E08DE00E94A129A4
:1045200061E08CE00E94A12960E08BE00E94A1295B
:1045300060E085E00E94A12961E085E00E94DA291F
:1045400060E086E00E94A12961E086E00E94DA290D
:1045500060E083E00E94A12961E083E00E94DA2903
:1045600061E08EE00E94A12960E08EE00E94DA29DD
:104570000E949F0740E052EC61E070E080EE95E021
:104580000E943C2D0E94A9130E94480D0E94921384
:104590008FEF8093A8040E94C60778940E94E828B1
:1045A0006B017C018091A8048F3F59F40E94E82898
:1045B0006C197D098E099F09603D77408105910541
:1045C00088F380ED97E00E94A80761E08BE00E94ED
:1045D000DA292D9A80EE95E00E94F42B892B29F0A0
:1045E00080EE95E00E94212CF5CF6DEF72E080EE19
:1045F00095E00E94AF2A83E893E00E94300C64E1CA
:1046000073E080EE95E00E94AF2A4AE050E062E05D
:1046100070E080EE95E00E947F2B62E370E080E026
:1046200090E00E94172980EE95E00E94F42B0497F9
:104630000CF180EE95E00E94212C82349105D1F49A
:1046400080EE95E00E94212C8E34910599F480EE45
:1046500095E00E94212C8434910561F480EE95E070
:104660000E94212C819731F480E090E00E94A807FD
:104670000E9448214091750550917605609177051B
:1046800070917805DB01CA010197A109B10904976E
:10469000A105B10568F44093A704433029F440EA2A
:1046A00056E861E070E004C040E052EC61E070E088
:1046B00080EE95E00E943C2D0E94DD212D9880E047
:1046C00090E00E94A8070E9492131092C304809168
:1046D000BD0583FF11C080918905882351F0809129
:1046E0009005882331F080919705882311F087E0A9
:1046F00001C085E08093C30480E00E947E0A80911F
:10470000C4040E94B2090E94590B10923F041092F7
:104710003E0410923D04F12C8091D2058F15B0F02B
:1047200062E370E080E090E00E94172980ED97E05E
:104730000E94A80762E370E080E090E00E941729E1
:1047400080E090E00E94A807F394E6CF80919C055A
:1047500084FF08C0982F987181E0983109F080E0BB
:104760000E947C118FE00E94DA07FF90EF90DF90AB
:10477000CF900895EF92FF920F931F93CF93DF9303
:104780008C016EE770E080EE95E00E945906E8012A
:10479000F12CF0E2EF2E8E0188818D57823048F4A3
:1047A0006DE770E080EE95E00E94590688818E25C5
:1047B00088832196F801608180EE95E00E944E2C5E
:1047C000F394F9E0FF12E7CF6EE770E080EE95E03A
:1047D0000E945906CDB7DEB7E6E00C94B52EA9E0ED
:1047E000B0E0E5EFF3E20C949D2E9091C504911199
:1047F0000EC09EEF99838A836B8350E05595479551
:104800004C832D83198618861F821E822EC04091EC
:10481000CA04842F90E0B4E095958795BA95E1F7A6
:10482000242F2F7030E08217930719F18DEF8983C1
:104830001B82FE01349650E0842F90E0A4E0959511
:104840008795AA95E1F7242F2F7030E08217930700
:1048500049F0DC01A553BB4F8C918193405F5F5FB2
:10486000563051F74093CA045A83CE0101960E94F4
:10487000BA238091C50490E0019666E070E00E9442
:10488000382E8093C5042996E2E00C94B92EA0E05E
:10489000B0E0EDE4F4E20C94962E6C016EE770E06B
:1048A00080EE95E00E9459068601E12CF12CC0E0D3
:1048B000D0E030E2B32EF801608183E8860F8230C9
:1048C00078F46DE770E080EE95E00E945906F801FB
:1048D00060816B2570E080EE95E00E94590604C06F
:1048E00080EE95E00E944E2CE114F10459F0F8019D
:1048F00080819E01280F311DC901C92FDD27C80FF6
:10490000D91FDD273FEFE31AF30A89E0E816F10427
:1049100059F028E0E216F10421F48C2F8095F6017D
:1049200080870F5F1F4FC7CFCDB7DEB7E9E00C948C
:10493000B22EA9E0B0E0EFE9F4E20C949D2EE82F4E
:10494000362F8091C50490E0019664E270E00E94E9
:10495000382E8093C50458E9598350E15A83813039
:1049600089F048F08230B9F08330D9F48B8381EF3D
:104970008C833D8319C085E08B8381EF8C832F5F0F
:104980002D8312C08B8381EF8C8384E6489FA00126
:1049900011245D8309C084E08B8381EF8C83ED83D8
:1049A00003C00E94B91104C0CE0101960E944724A1
:1049B0002996E2E00C94B92EA2E0B0E0E2EEF4E237
:1049C0000C94922E182F762E2A8349830E94F42865
:1049D0006B017C018091DB048090C6049090C70439
:1049E000A090C804B090C9042A8149818823C1F0ED
:1049F000D701C60188199909AA09BB094C015D01B3
:104A000091EE89169EE29906A104B10420F12417C3
:104A100008F4422F202F672D812F0E94992413C064
:104A2000D701C60188199909AA09BB094C015D0182
:104A300091E3891695E79906A104B10460F0672D0A
:104A4000812F0E94EF23C092C604D092C704E09247
:104A5000C804F092C9042296EDE00C94AE2EA2E2B6
:104A6000B0E0E5E3F5E20C94932E8CE00E94990906
:104A700081110DC06CE173E080EE95E00E94E02AA8
:104A80002D9A80E00E947E0A0E94590B2D9880EE9C
:104A900095E00E94F42B892B01F180EE95E00E94B5
:104AA000212C9091A704992319F00E94E513EFCFD0
:104AB00040913E0450E09A012F5F3F4F2F71332702
:104AC00060913F0470E02617370709F3FA01E75BAE
:104AD000FB4F808320933E04DACF809171058430B0
:104AE00009F086C00E94F4286115710581059105C1
:104AF00049F06093B5047093B6048093B704909323
:104B0000B8040CC081E090E0A0E0B0E08093B50470
:104B10009093B604A093B704B093B8048091AB040B
:104B20009091AC0481609093AC048093AB0483E0DB
:104B3000809371058FE70E94770909E614E00E94CF
:104B40008A09F80181938F01F4E002371F07B9F752
:104B50002091720480916904982F922796FF3BC0A0
:104B600090E4922790937204982F98739833F1F4FD
:104B700010E0212F30E080916904877090E0821767
:104B800093074CF11F5F20919C05812F90E0FC0161
:104B9000E759FB4F24FF04C080810E949B11E9CF9D
:104BA000608180EE95E00E944E2CE3CF8F7399F4E4
:104BB00080916A048093B40480916B048093B20462
:104BC00080916C048093B10480916F0490E0909385
:104BD000AA048093A90480913D04813019F482E0F5
:104BE00080933D0480913D04833011F410923D0484
:104BF0000E94F4286B017C018091AD049091AE0479
:104C0000A091AF04B091B0040097A105B105C9F01F
:104C1000A7019601281B390B4A0B5B0BDA01C9016E
:104C2000883B9B40A105B10560F00E94C8098093B4
:104C3000B3041092AD041092AE041092AF0410921F
:104C4000B0048091B9049091BA04A091BB04B091D2
:104C5000BC0446015701881A990AAA0ABB0A84E7CC
:104C600095E00E94F40786169706A806B90608F490
:104C7000B1C0C092B904D092BA04E092BB04F092E1
:104C8000BC040E9457068091A8048830A0F080914F
:104C9000BD059091BE05A091BF05B091C0055CE136
:104CA000B695A795979587955A95D1F7892B8A2B15
:104CB0008B2B09F0B8C18091A8048F5F8093A80462
:104CC0008091B5049091B604A091B704B091B80456
:104CD0000097A105B105F1F0C81AD90AEA0AFB0A42
:104CE00084E795E00E94F4076C157D058E059F050D
:104CF00008F00FC18091BD0584FD04C080ED97E0F0
:104D00000E94A8071092B5041092B6041092B7043E
:104D10001092B80490917204907C90937204509118
:104D20003E0480913F0420913D04581709F40EC1C0
:104D3000223009F00BC1905890937204E0919C05C9
:104D4000E770F0E0E658FC4F6081693008F0E6C09B
:104D5000615040E04613E4C080933F0487E3840F32
:104D600090917204892B809372044093400483E0F5
:104D700080933D042C9A109181058091C304811188
:104D800032C18091BD0582FD3AC1812F0E94790A0E
:104D90008091C4040E94B209E0919C05E770F0E0A4
:104DA000E658FC4F608182E794E00E94940B80916A
:104DB000BD0582FD2DC1E091C404EF5FE093C40402
:104DC000E83109F42DC1F0E0EC58FA4F87858823CB
:104DD00009F426C10E94030C813069F580919C057D
:104DE000887149F18091AB049091AC04880F991FB0
:104DF0009093AC048093AB0483E0809371050E9490
:104E0000590B0E94F4286093AD047093AE04809314
:104E1000AF049093B004672B682B692B61F481E099
:104E200090E0A0E0B0E08093AD049093AE04A09336
:104E3000AF04B093B00480919C0584FF1FC08091A3
:104E4000AB049091AC048E7F0E942A09182F6091C8
:104E5000A9048091B4040E94DB13482F612F809134
:104E6000B30449A30E94DB130091D205282F49A166
:104E70006091B1048091B2040E94DC242C9880914E
:104E8000C1048130C1F018F08230B1F1D9C08BE09B
:104E90000E940D2A892B09F0D3C081E08093C104C0
:104EA0000E94E8286093BD047093BE048093BF0401
:104EB0009093C004C5C08BE00E940D2A892B31F568
:104EC0000E94E828C090BD04D090BE04E090BF04CA
:104ED000F090C0046C197D098E099F09693E7340EA
:104EE0008105910508F4ACC082E08093C10480ED97
:104EF00097E00E94A807A4C08BE00E940D2A892B8E
:104F000009F49EC080E090E00E94A8071092C104BE
:104F100097C080E090E00E94A807FCCE68E019CF1F
:104F2000851709F419CF4F5F242F30E090E0F90185
:104F3000EE58FB4FDC01A75BBB4F7C917083F901FE
:104F4000E05CFB4F708301968F7104CF2430B1F485
:104F50002091400481E494E0A3E7B4E0FC013E2FFB
:104F6000381B321718F431913D93F9CF87E3820F44
:104F700090917204892B80937204F9CE8091C104C0
:104F8000823051F49160909372042D9A8E010F5FDC
:104F90001F4FF12CB80110C02D9880913D04811154
:104FA00003C081E080933D0480913D04833071F71C
:104FB00084E080933D04EACF8F2D69A37AA30E94F9
:104FC000DD15F801819391938F01F39469A17AA182
:104FD000F0E1FF12F1CF80919C0543E754E0877028
:104FE0000E947908C7CE112309F4CBCE9091C20458
:104FF00021E0290F2093C2049813C3CE1DC085E081
:105000000E940D2A892B09F0C0CE2D9A17E0BDCE43
:1050100085E00E940D2A892B09F0CDCE2D98CBCEAC
:105020001092C404D7CE8091A804883009F42D9A38
:1050300089E08093A804CECE1092C2041150A1CE74
:10504000A296ECE00C94AF2E8230E8F4E82FF0E06A
:10505000EE0FFF1FED52FA4F71836083813041F0F4
:10506000809169008C7F842B80936900E89A089571
:1050700080916900440F551F440F551F837F842B77
:1050800080936900E99A08951F920F920FB60F92CC
:1050900011242F933F934F935F936F937F938F933D
:1050A0009F93AF93BF93EF93FF938091D30590911C
:1050B000D405892B29F0E091D305F091D405099509
:1050C000FF91EF91BF91AF919F918F917F916F91E0
:1050D0005F914F913F912F910F900FBE0F901F90B6
:1050E00018951F920F920FB60F9211242F933F9392
:1050F0004F935F936F937F938F939F93AF93BF93E0
:10510000EF93FF938091D5059091D605892B29F0D7
:10511000E091D505F091D6050995FF91EF91BF91EA
:10512000AF919F918F917F916F915F914F913F913F
:105130002F910F900FBE0F901F9018951F920F92F6
:105140000FB60F9211242F933F938F939F93AF939A
:10515000BF938091D8059091D905A091DA05B091BF
:10516000DB053091D70523E0230F2D3720F401967E
:10517000A11DB11D05C026E8230F0296A11DB11D7A
:105180002093D7058093D8059093D905A093DA058D
:10519000B093DB058091DC059091DD05A091DE05E3
:1051A000B091DF050196A11DB11D8093DC059093A0
:1051B000DD05A093DE05B093DF05BF91AF919F9110
:1051C0008F913F912F910F900FBE0F901F901895C8
:1051D0002FB7F8946091D8057091D9058091DA05C0
:1051E0009091DB052FBF08953FB7F8948091DC05BF
:1051F0009091DD05A091DE05B091DF0526B5A89B55
:1052000005C02F3F19F00196A11DB11D3FBF6627B4
:10521000782F892F9A2F620F711D811D911D42E0F9
:10522000660F771F881F991F4A95D1F70895CF926F
:10523000DF92EF92FF92CF93DF936B017C010E948C
:10524000F428EB01C114D104E104F10479F00E94C7
:10525000F4286C1B7D0B683E7340A0F381E0C81AF4
:10526000D108E108F108C851DC4FECCFDF91CF91B4
:10527000FF90EF90DF90CF900895789484B582608E
:1052800084BD84B5816084BD85B5826085BD85B5EA
:10529000816085BDEEE6F0E0808181608083E1E899
:1052A000F0E01082808182608083808181608083D1
:1052B000E0E8F0E0808181608083E1EBF0E08081D4
:1052C00084608083E0EBF0E0808181608083EAE7A6
:1052D000F0E080818460808380818260808380812F
:1052E000816080838081806880831092C1000895EE
:1052F000833081F028F4813099F08230A1F0089554
:105300008630A9F08730B9F08430D1F480918000E4
:105310008F7D03C0809180008F77809380000895F7
:1053200084B58F7702C084B58F7D84BD0895809148
:10533000B0008F7703C08091B0008F7D8093B00064
:105340000895CF93DF9390E0FC01ED50F44F24914A
:10535000FC01E95FF34F8491882349F190E0880FC5
:10536000991FFC01E15DF34FA591B4918B5D934FC3
:10537000FC01C591D4919FB7611108C0F8948C913C
:10538000209582238C93888182230AC0623051F455
:10539000F8948C91322F309583238C938881822BC3
:1053A000888304C0F8948C91822B8C939FBFDF91EB
:1053B000CF910895A1E0B0E0E0EEF9E20C949B2ECD
:1053C000282F30E0F901E152F44F8491F901ED50BA
:1053D000F44F1491F901E95FF34F04910023C9F0F0
:1053E000882321F069830E9478296981E02FF0E009
:1053F000EE0FFF1FEB5DF34FA591B4919FB7F894AB
:105400008C91611103C01095812301C0812B8C9375
:105410009FBF2196E4E00C94B72ECF93DF93282F03
:1054200030E0F901E152F44F8491F901ED50F44F6D
:10543000D491F901E95FF34FC491CC2391F081112C
:105440000E947829EC2FF0E0EE0FFF1FE55EF34F8E
:10545000A591B4912C912D2381E090E021F480E07E
:1054600002C080E090E0DF91CF9108958E3008F087
:105470008E50877020919D0190E4299F9001112406
:10548000822B80937C0080917A00806480937A00E4
:1054900080917A0086FDFCCF809178002091790080
:1054A00090E0922B0895A0E0B0E0E9E5FAE20C94D8
:1054B000972E6C017A01EB01E60EF71E00E010E07A
:1054C000CE15DF0561F06991D601ED91FC91019057
:1054D000F081E02DC6010995080F191FF1CFC80111
:1054E000CDB7DEB7E8E00C94B32E6115710589F0F5
:1054F000DB010D900020E9F7AD0141505109461B39
:10550000570BDC01ED91FC910280F381E02D0995B0
:10551000089580E090E00895EF92FF920F931F931B
:10552000CF93DF938C01FB01C0E0D0E064917F0159
:105530008FEFE81AF80A662361F0D801ED91FC912B
:105540000190F081E02DC8010995C80FD91FF7011E
:10555000EDCFCE01CDB7DEB7E6E00C94B52E0E94BC
:10556000752A0895DC01ED91FC910190F081E02D08
:10557000099508950F931F93CF93DF93EC016DE08E
:105580000E94B22A8C016AE0CE010E94B22A800FEA
:10559000911FDF91CF911F910F9108950F931F934A
:1055A000CF93DF93EC010E948C2A8C01CE010E94E4
:1055B000BA2A800F911FDF91CF911F910F9108950B
:1055C0000F931F93CF93DF93EC010E94752A8C01F8
:1055D000CE010E94BA2A800F911FDF91CF911F91B7
:1055E0000F9108950F931F93CF93DF93EC010E94C7
:1055F000B22A8C01CE010E94BA2A800F911FDF913E
:10560000CF911F910F910895A1E2B0E0EAE0FBE293
:105610000C94932E7C01C42EE52FCB01D22E19A21F
:1056200021E02D1510F02AE0D22E8E010F5D1F4FC4
:105630008D2C912CA12CB12C6C2D7E2FA5019401C9
:105640000E944C2E8C2DD29E8019112401501109DC
:105650008A3010F4805D01C0895CF80180832115D7
:1056600031054105510521F0C22EE32FCA01E4CFD7
:10567000B801C7010E94752AA196ECE00C94AF2EE8
:10568000A0E0B0E0E6E4FBE20C94972EEC016A01A6
:105690007B012115310541F4E881F9810190F08108
:1056A000E02D642F09951DC02A303105A9F477FF3C
:1056B00012C06DE20E94B22A8C0144275527BA011C
:1056C0004C195D096E097F092AE0CE010E94042B66
:1056D000800F911F06C02AE0B701A601CE010E94EB
:1056E000042BCDB7DEB7E8E00C94B32E9A01AB01E2
:1056F000662757FD6095762F0E94402B08950F93E3
:105700001F93CF93DF93EC019A01AB01662757FDFE
:105710006095762F0E94402B8C01CE010E94BA2A00
:10572000800F911FDF91CF911F910F910895211547
:10573000310549F4DC01ED91FC910190F081E02DFF
:10574000642F099508950E94042B08959A01462F0D
:1057500050E060E070E00E94972B08959A01AB0141
:1057600060E070E00E94972B08950F931F93CF93F2
:10577000DF93EC010E94972B8C01CE010E94BA2A84
:10578000800F911FDF91CF911F910F9108950F937B
:105790001F93CF93DF93EC019A01AB0160E070E0BF
:1057A0000E94972B8C01CE010E94BA2A800F911F74
:1057B000DF91CF911F910F9108950F931F93CF9376
:1057C000DF93EC019A01462F50E060E070E00E9408
:1057D000972B8C01CE010E94BA2A800F911FDF9176
:1057E000CF911F910F910895FC0124853585F90112
:1057F000E05CFF4F80819181F901EE5BFF4F2081DA
:105800003181821B930B8F7399270895FC01848546
:105810009585FC01E05CFF4F40815181FC01EE5B0E
:10582000FF4F208131814217530741F00190F081F1
:10583000E02DE80FF91F808190E008958FEF9FEF32
:105840000895FC0184859585FC01E05CFF4F408153
:105850005181FC01EE5BFF4F2081318142175307DC
:1058600079F0A081B181A80FB91F8C91208131817D
:105870002F5F3F4F2F7333273183208390E00895AC
:105880008FEF9FEF0895FC0181A1882329F0A4895F
:10589000B5898C9186FFFBCF11A20895CF93DF933A
:1058A000FC0126853785D901A05CBF4F8D919C9165
:1058B000119701968F739927E901CE5BDF4F4881DD
:1058C000598184179507D9F30D90BC91A02DA20F93
:1058D000B31F6C93A685B785A05CBF4F11969C93B0
:1058E0008E93A689B7892C9181E090E0078C02C045
:1058F000880F991F0A94E2F7282B2C9381E081A34B
:105900000488F589E02D80818064808381E090E0C7
:10591000DF91CF91089508951F920F920FB60F92C5
:1059200011242F933F934F938F939F93EF93FF9364
:105930008091C00082FD1CC04091C6008091860607
:105940009091870601968F73992720918806309150
:1059500089068217930771F0E0918606F091870619
:10596000EA5BF94F4083909387068093860602C0D6
:105970008091C600FF91EF919F918F914F913F9140
:105980002F910F900FBE0F901F90189580EE95E00D
:105990000E94F42B892B11F00E948B2C08951F92EA
:1059A0000F920FB60F9211242F933F938F939F93D3
:1059B000EF93FF9320914206309143068091440675
:1059C000909145062817390731F48091C1008F7DE9
:1059D0008093C10014C0E0914406F0914506EE5F4B
:1059E000F94F2081809144069091450601968F736E
:1059F000992790934506809344062093C600FF9113
:105A0000EF919F918F913F912F910F900FBE0F902B
:105A10001F901895A0E0B0E0E0E1FDE20C94932E19
:105A2000FC011382128288EE93E0A0E0B0E0848350
:105A30009583A683B7838CEB93E0918380837587EE
:105A4000648757874687318B208B138B028BF58AAF
:105A5000E48AD78AC68AB18EA08E938E828E8F8575
:105A6000848F8889858F8989868F8A89878F8B899A
:105A700080A3ECE00C94AF2ECF92DF92EF92FF92D6
:105A8000CF93DF93EC016A017B01411581EE58074A
:105A900061057105F9F0EC89FD8981E090E008A0CD
:105AA00002C0880F991F0A94E2F7808360E079E0D2
:105AB0008DE390E0A70196010E944C2E2150310900
:105AC000410951095695479537952795211580E14C
:105AD000380798F0EC89FD89108260E874E88EE15F
:105AE00090E0A70196010E944C2E215031094109F6
:105AF00051095695479537952795E889F989308357
:105B0000EA89FB89208319A2EE89FF89408181E01F
:105B100090E09C010C8C02C0220F331F0A94E2F724
:105B2000422B4083EE89FF8940819C010D8C02C08D
:105B3000220F331F0A94E2F7422B4083EE89FF893C
:105B400040819C010E8C02C0220F331F0A94E2F7A1
:105B5000422B4083EE89FF8920810F8C02C0880F81
:105B6000991F0A94E2F7809582238083DF91CF9179
:105B7000FF90EF90DF90CF9008958F929F92AF9219
:105B8000BF92CF92DF92EF92FF920F931F9381E02B
:105B90008F9385E08F9387E08F9383E08F9384E0EA
:105BA0008F93E6EC8E2E912CF2ECAF2EB12CA1EC63
:105BB000CA2ED12CB0ECEB2EF12C04EC10E025EC2D
:105BC00030E042E056E066E476E080EE95E00E9448
:105BD0000A2D0F900F900F900F900F901F910F9123
:105BE000FF90EF90DF90CF90BF90AF909F908F90FD
:105BF00008950E943D290E948322C6ECDCE20E94A7
:105C00002F252097E1F30E94C62CF9CFA29FB00167
:105C1000B39FC001A39F700D811D1124911DB29FE0
:105C2000700D811D1124911D08950E94062EA59FBF
:105C3000900DB49F900DA49F800D911D1124089587
:105C4000B7FF0C94152E0E94152E821B930B0895FE
:105C5000DB018F939F930E94152EBF91AF91A29F5E
:105C6000800D911DA39F900DB29F900D112408955A
:105C700097FB072E16F4009407D077FD09D00E94F9
:105C8000CA2E07FC05D03EF4909581959F4F08954C
:105C9000709561957F4F0895A1E21A2EAA1BBB1B38
:105CA000FD010DC0AA1FBB1FEE1FFF1FA217B307E8
:105CB000E407F50720F0A21BB30BE40BF50B661FFE
:105CC000771F881F991F1A9469F7609570958095C2
:105CD00090959B01AC01BD01CF010895052E97FB66
:105CE0001EF400940E94852E57FD07D00E944C2E72
:105CF00007FC03D04EF40C94852E509540953095BA
:105D000021953F4F4F4F5F4F089590958095709527
:105D100061957F4F8F4F9F4F08952F923F924F92E3
:105D20005F926F927F928F929F92AF92BF92CF922B
:105D3000DF92EF92FF920F931F93CF93DF93CDB734
:105D4000DEB7CA1BDB0B0FB6F894DEBF0FBECDBFAC
:105D500009942A88398848885F846E847D848C847D
:105D60009B84AA84B984C884DF80EE80FD800C8186
:105D70001B81AA81B981CE0FD11D0FB6F894DEBF69
:105D80000FBECDBFED010895EE0FFF1F0590F491FA
:105D9000E02D0994AA1BBB1B51E107C0AA1FBB1F22
:105DA000A617B70710F0A61BB70B881F991F5A95A7
:105DB000A9F780959095BC01CD0108958F929F928F
:105DC000AF92BF92CF92DF92EF92FF92CF93DF9389
:105DD000EC01688179818A819B816115710581055A
:105DE000910521F464E279ED8BE597E02DE133EF45
:105DF00041E050E00E946E2E49015A019B01AC0126
:105E0000A7EAB1E40E94152E6B017C01ACEEB4EF61
:105E1000A50194010E94232EC60ED71EE81EF91E6E
:105E2000F7FE06C081E0C81AD108E10880E8F80A48
:105E3000C882D982EA82FB82C701B6019F77DF91CF
:105E4000CF91FF90EF90DF90CF90BF90AF909F9059
:105E50008F9008950E94DE2E089586E091E00E94C2
:105E6000DE2E089560930601709307018093080168
:105E70009093090108952F923F925F926F927F92C3
:105E80008F929F92AF92BF92CF92DF92EF92FF924A
:105E90000F931F93CF93DF938B01EA016115710577
:105EA00021F0DB018C9311969C93209739F09E0191
:105EB000225031092332310508F0D8C07C01670136
:105EC000BFEFCB1ADB0A5601F7016080862D90E008
:105ED0000E946D30892B11F07601F1CFFDE26F1237
:105EE0000AC0570182E0A80EB11CD70111966C9030
:105EF000772473940BC0BBE26B1207C05701E2E03A
:105F0000AE0EB11CD70111966C90712CCE018F7E14
:105F1000892B89F4B0E36B1237C0F50180818F7D46
:105F20008835D1F46180F2E0AF0EB11C872D82601C
:105F3000782EC0E1D0E0CA30D10551F1C031D10591
:105F400021F0C830D10599F409C0CC24CA94DC2CC6
:105F5000EC2CAFE0FA2E22C0209769F7C8E0D0E021
:105F6000CC24CA94DC2CEC2CFFE1FF2E17C06FEF81
:105F70007FEFCB019E01442737FD4095542F0E94AF
:105F80004C2E69017A010AC02097A9F6CAE0D0E038
:105F9000E9E9CE2EDC2CEC2CE9E1FE2EF50160E0E7
:105FA00020E030E0A9014E01AA2497FCA094BA2C6D
:105FB0001F0170ED572E560CA9E0A51570F48FEB5C
:105FC000860D8A3118F499EC592E06C08FE9860D9A
:105FD0008A3148F589EA582E560C852D90E08C17A9
:105FE0009D070CF56F3FD9F0C216D306E406F506FF
:105FF00098F0C501B4010E94282E9B01AC01852DAB
:1060000090E0A0E0B0E0280F391F4A1F5B1F28175F
:1060100039074A075B0710F46FEF01C061E0319662
:10602000D1016C90C5CF0115110551F0662311F017
:10603000319703C071FE04C03297D801ED93FC93F1
:1060400070FE07C050954095309521953F4F4F4FBA
:106050005F4F67FF10C082E290E090938B068093C1
:106060008A066FEF7FEF8FEF9FEF07C060E070E071
:1060700080E090E002C0B901CA01DF91CF911F9189
:106080000F91FF90EF90DF90CF90BF90AF909F90D7
:106090008F907F906F905F903F902F900895FC01BC
:1060A00088279927E89421912032E9F3293010F0CC
:1060B0002E30C8F32B3241F02D3239F4689404C0ED
:1060C0000E94A130820F911D219120532A30C0F3EC
:1060D0001EF4909581959F4F0895911150C0803284
:1060E00019F089508550D0F7089548EC53E00E948C
:1060F0007A300895FA01A191B081009719F41097B0
:10610000E1F0CD01DC01CD010D90002011F4C001C2
:1061100013C0FB012191222319F02015D9F7F3CFE9
:10612000FB012191201519F41E92119606C022231D
:10613000C1F70D900020A1F7D001FA01A193B0831F
:1061400008957AE0979F902D879F802D910D1124BF
:106150000895F999FECF92BD81BDF89A992780B52F
:106160000895262FF999FECF1FBA92BD81BD20BD9B
:106170000FB6F894FA9AF99A0FBE019608959927E6
:0861800088270895F894FFCF71
:1061880000008C06200001000000FF000200020051
:1061980002000200020002000200020002000200E7
:1061A8000200020002000200020002802500000531
:1061B800400AA1204EA50020244EA52C2330C01251
:1061C80000001A400AA1204EA5001B1E27522C23AE
:1061D800308025000005400AA1204EA50020244E4D
:1061E800A52C2330004B000006400AD0009D490032
:1061F8007B289D492C233000E1000005400A450119
:10620800D7DC03B81E0EBF00232E48E801008A40E1
:106218000A6001555502AD1E20000023C8015458DC
:106228002074696D656F75742100596573004E6F30
:10623800002C00386368004E2F41002C205B005D65
:106248002028002900486F70206368616E6E656CB5
:10625800200020402000456E746572696E672061D9
:1062680064617074697665206368616E6E656C2020
:1062780073656C656374696F6E2C207069636B69F4
:106288006E673A007363616E6E6572206D6F646548
:10629800004E4F5420454E41424C45440053656ED4
:1062A80064696E672073657474696E677320746FB0
:1062B8002052580A00526573657474696E672073BA
:1062C800657474696E6773206F6E2052580A0041B6
:1062D800626F727465642065646974730A00696E1C
:1062E80076616C69642073656C656374696F6E00B0
:1062F8000D0A496E76616C696420696E7075742048
:106308002D206469736361726465642107005365B5
:106318007474696E677320736176656420746F2086
:10632800454550524F4D0A00526576657274656452
:106338002073657474696E67732066726F6D20458B
:106348004550524F4D0A004C6F6164656420666188
:1063580063746F72792064656661756C74730A0082
:106368004B657920616E64206368616E6E656C733D
:106378002072616E646F6D697A65640A004F70659A
:106388006E4C52536E67205458207374617274694E
:106398006E672000206F6E20485720006D6F64756F
:1063A8006C65206C6F636B65643F00342B34003878
:1063B80000382B340031320031322B3400313600B2
:1063C80050504D0052535349005344410053434CDD
:1063D80000525844005458440041494E004C42452C
:1063E80045500053504B54524D005342555300539F
:1063F800554D44004C4C494E440000070B0C1011FD
:106408001500B7012B032F033103350338033D0370
:10641800B7014003440349034D035103550359038E
:106428005D0363036A036F0374038D028D028D029B
:106438008D02160A13223129000000004E2C532A1F
:08644800F42B212C062C432C3F
:00000001FF
